:04000000B6010D290F
:1000080008009818181218162C08A0002D08A1002E
:10001800A201A3010F28102864008C1A2C28FF3095
:10002800A207031CA307031CA007031CA107031CAA
:100038000829220F0E28230F0F28FA30A2000030BB
:10004800A300102898181812181664008C1E292866
:100058001A080314082964000C1E2F289900031499
:100068000829B616B61EB612B6193E28B615772058
:10007800031865280830A3008B20A20DA30B402885
:10008800B61E702095209120B61A65206A20220895
:1000980003100829B616B61EB61236195828FE39A6
:1000A800B700361503100829361A6028A600361638
:1000B80077200318652826087E2003186528B61EB1
:1000C80008297020952036113612B6113A08840096
:1000D80038088417800476283A088400380980058F
:1000E8008417800508006A20952070209120370821
:1000F800B6190138A2000830A300A20D03186A201F
:10010800031C702095209120A30B81286A2095203C
:100118003A08840038080005FF3E3B088400390986
:1001280073283B08840039086D28A40029080314A3
:10013800031908290321031C0800A00025188317A8
:1001480024088400200880008313A40AA9039A289D
:1001580083178001840AFF3E031DAD280829A301E7
:10016800A200FF30A207031CA307031C08290330C1
:10017800A100E630C120B528A101FC3EA000A109DC
:10018800031CCC28FF300000A0070318C728A007CD
:100198006400A10FC62808000310A00DA10DFF3EA2
:1001A8000318D02820080829A2000130DD28A20061
:1001B8000530A80023082102031DE4282208200294
:1001C800043003180130031902302805031DFF30DD
:1001D80008291030A800A101A001A70CA60C031C37
:1001E800FB282208A00723080318230FA107A10C46
:1001F800A00CA50CA40CA80BF1282408082984003D
:1002080031088A00300882008313031383126400C4
:10021800080083160F309900203098008312903020
:1002280098002030840060308A01AD20A03084001E
:1002380050308A01AD201030840060308A01AC2033
:100248009030840060308A01AC20831607309F000C
:10025800D701D801861006118801071087100711E9
:1002680083120711861001308A01B3208614643086
:100278008A01B32053308A012F2074308A012F203D
:1002880061308A012F2072308A012F2074308A0150
:100298002F2069308A012F206E308A012F20673085
:1002A8008A012F202E308A012F202E308A012F20FC
:1002B8008A110A12722B07108316420883128800CB
:1002C8008A110A126C2907148316440883128800BD
:1002D8008710000087140710080083164630C400F2
:1002E80083128A0167218316C20183128A015F2162
:1002F80083161030C20083128A015F2183164C30A6
:10030800C40083128A01672183164230C400831215
:100318008A0167218316C2010130C6008312640076
:100328008130831646028A110A1283120318B929EA
:1003380083160130C90083126400213083164902F4
:100348008A110A1283120318B2298A015F218316BF
:10035800C90A8A110A128312031DA0298316C60A24
:100368008A110A128312031D932983164630C4008A
:1003780083128A0167218316C20183128A015F21D1
:1003880083161030C20083128A015F2183164C3015
:10039800C40083128A016721080083164630C4000E
:1003A80083128A0167218316C20183128A015F21A1
:1003B80083161030C20083128A015F2183164C30E5
:1003C800C40083128A016721080083164630C400DE
:1003D80083128A0167218316C20183128A015F2171
:1003E8008316C20183128A015F2183164C30C40030
:1003F80083128A01672183164230C40083128A015E
:10040800672183160130C6008312640011308316F9
:1004180046028A110A1283120318332A83160130FE
:10042800C900831264002130831649028A110A1216
:10043800831203182C2A83162030C20083128A01E3
:100448005F218316C90A8A110A128312031D162A0C
:100458008316C60A8A110A128312031D092A8316F3
:100468004630C40083128A0167218316C2018312B1
:100478008A015F218316C2014C30C40083128A01AD
:100488006721080083164030C40083128A0167215F
:100498008316C601831264000830831646028A1147
:1004A8000A1283120318802A83164608073C8A1109
:1004B8000A128312031C772A8A110A1269228316E8
:1004C800C20083128A110A12772A02308A00831620
:1004D8004608831282073034873407341F34523475
:1004E8007F34203400348A015F218316C60A8A11BA
:1004F8000A128312031D4F2A83164430C400831244
:100508008A0167218316C6018312640006308316A8
:1005180046028A110A1283120318B82A831646085B
:10052800053C8A110A128312031CAF2A8A110A1287
:10053800A3228316C20083128A110A12AF2A02303C
:100548008A008316460883128207003400347F34F9
:10055800003410347F348A015F218316C60A8A1159
:100568000A128312031D892A83165A30C400831283
:100578008A0167218316C20183128A015F218316CB
:100588005B30C40083128A01672183160130C200E0
:1005980083128A015F2183165830C40083128A01AE
:1005A800672183161630C20083128A015F218A01EF
:1005B80071218A01E92183164630C40083128A0119
:1005C80067218316C20183128A015F218316C20143
:1005D80083128A015F2183164C30C40083128A017A
:1005E800672183164230C20083128A015F21831675
:1005F800C20183128A015F2183165D30C400831211
:100608008A01672183160430C20083128A015F21A0
:1006180083168630C20083128A015F2183165930FF
:10062800C40083128A01672183161430C200831222
:100638008A015F2183164C30C40083128A01672126
:100648000800831646083C3E840000088312B20066
:10065800FF30A200A20A22080F3C8A110A12031CCA
:10066800582B8A110A12442332028A110A12031DD6
:100678002E2B22088316CE0083128A110A12582BB9
:1006880003308A002208820730343134323433345C
:1006980034343534363437343834393441344234E8
:1006A8004334443445344634080083164630C40085
:1006B80083128A01672183162A08C20083128A01DD
:1006C8005F2183162B08C20083128A015F218316DB
:1006D8004508C40083128A01672108008A0146225E
:1006E8008316A530AA00AB014C30C50083128A01DD
:1006F800592383164230C40083128A016721831666
:10070800C601831264001630831646028A110A1243
:1007180083120318C52B83164608153C8A110A1242
:100728008312031CBC2B8A110A12A0238316C20051
:1007380083128A110A12BC2B03308A0083164608DA
:1007480083128207503449344334203443346F349D
:100758006E34743472346F346C346C34653464348D
:10076800203453344534443431343334333430341E
:100778008A015F218316C60A8A110A128312031D91
:10078800862B8316C630AA00AB014C30C5008312F5
:100798008A01592383164230C40083128A016721D3
:1007A8008316C601831264001330831646028A1129
:1007B8000A12831203181D2C83164608123C8A114C
:1007C8000A128312031C142C8A110A12F1238316AD
:1007D800C20083128A110A12142C04308A0083166C
:0607E80046088312002CFC
:100800008207323435343634783431343234383443
:10081000203447347234613470346834693463345A
:1008200020344C34433444348A015F218316C60A91
:100830008A110A128312031DD72B8316E330AA00F4
:10084000AB014C30C50083128A0159238316423014
:10085000C40083128A0167218316C60183126400D3
:100860001B30831646028A110A1283120318732C56
:10087000831646081A3C8A110A128312031C6A2C3A
:100880008A110A1249248316C20083128A110A129D
:100890006A2C04308A008316460883128207553476
:1008A000733469346E3467342034503469346334BB
:1008B00042346134733469346334503472346F3485
:1008C00020345634653472342E34203432342E348D
:1008D000343432348A015F218316C60A8A110A121F
:1008E0008312031D2F2C83160530AA000130AB00A4
:1008F0004C30C50083128A01592383164230C4004C
:1009000083128A0167218316C601831264001530A1
:10091000831646028A110A1283120318C42C831606
:100920004608143C8A110A128312031CBB2C8A113C
:100930000A12A0248316C20083128A110A12BB2C49
:1009400004308A00831646088312820752346134C9
:100950006E346A34693474342034443469346F3406
:100960006C3420342D34203443344F344D345034DF
:100970005334793473348A015F218316C60A8A118D
:100980000A128312031D862C83162430AA0001301C
:10099000AB004C30C50083128A01592383164230C4
:1009A000C40083128A0167218316C6018312640082
:1009B0001730831646028A110A1283120318212D5A
:1009C00083164608163C8A110A128312031C182D3E
:1009D0008A110A12F1248316C20083128A110A12A4
:0E09E000182D05308A00831646088312002D5C
:100A0000820768347434743470343A342F342F3499
:100A10007734773477342E3463346F346D347034F4
:100A200073347934733431342E3463346F346D3429
:100A30008A015F218316C60A8A110A128312031DD6
:100A4000D72C83168230AA000130AB004C30C50091
:100A500083128A01592383164230C40083128A010B
:100A600067218316C601831264001B308316460279
:100A70008A110A1283120318782D831646081A3C2D
:100A80008A110A128312031C6F2D8A110A124E2535
:100A90008316C20083128A110A126F2D05308A0054
:100AA0008316460883128207553473346534203424
:100AB0007734693474346834203447344C344334E4
:100AC0004434203454344F344F344C345334203471
:100AD000563465347234203431342E3434348A013F
:100AE0005F218316C60A8A110A128312031D342D50
:100AF0008316AA011030AB004F30C50083128A0163
:100B0000592383164230C40083128A016721831659
:100B10008030C200C6018312640080308316460212
:100B20008A110A12831203189E2D8A015F218316EF
:100B3000C60A8A110A128312031D8C2D83161F30D8
:100B4000AA001030AB004F30C50083128A01592330
:100B500083164230C40083128A0167218316013054
:100B6000C200C601831264008030831646028A11D7
:100B70000A1283120318C52D8A015F218316C60A43
:100B80008A110A128312031DB32D8316AA01103095
:100B9000AB004C30C50083128A01592383164230C2
:100BA000C40083128A0167218316FF30C200C60188
:100BB000831264002030831646028A110A128312BF
:100BC0000318EB2D8A015F218316C60A8A110A12C7
:100BD0008312031DD92D8316E030AA001F30AB000D
:100BE0004C30C50083128A01592383164230C40059
:100BF00083128A0167218316FF30C200C601831267
:100C000064002030831646028A110A1283120318E8
:100C1000122E8A015F218316C60A8A110A128312D4
:100C2000031D002E8316C901C601CA012030C10070
:100C3000AA01AB01B401B501B601B7017830C70014
:100C4000C801573083128A012F2061308A012F207A
:100C500069308A012F2074308A012F2069308A017F
:100C60002F206E308A012F2067308A012F202E30EE
:100C70008A012F202E308A012F200A308A012F204E
:100C80000D308A012F2011308A012F2011308A0166
:100C90002F2011308A012F208A012620403C8A1102
:100CA0000A12031D4C2E0B30A9002630B000B101F2
:100CB000A501A0308A01992013308A012F2013301A
:100CC0008A012F2013308A012F2013308A012F2010
:100CD0008A01E9218316C601831264000B30831652
:100CE00046028A110A1283120318B52E831646088B
:100CF000A03E840000088312B200FF30A200A20AC6
:100D000022080F3C8A110A12031CA92E8A110A120A
:100D1000952632028A110A12031D7F2E220883169D
:100D2000CE0083128A110A12A92E06308A002208E8
:100D30008207303431343234333434343534363459
:100D4000373438343934413442344334443445340C
:100D5000463483164608A03E84004E088000C60A2A
:100D60008A110A128312031D6D2E83162008C900F2
:100D700021088312A000A10104308A01D320B2000F
:100D80002108B30083162208831232048316C1009F
:100D900023088312A000A10104308A01D320B200ED
:100DA0002108B30083162408831232048316AB0093
:100DB00025088312A000A10104308A01D320B200CB
:100DC0002108B30083162608831232048316AA0072
:100DD00027088312A000A10104308A01D320B200A9
:100DE0002108B30083162808831232048316D0002A
:100DF00029088312A000A10104308A01D320B20087
:100E00002108B30083162A08831232048316CF0008
:100E10002B08D1002A08D2002A088312FE0083166C
:100E20002B088312FF00831650088312FD008316DF
:100E30004F088312FC00640083164908003C8A15A1
:100E40000A12831203196629640083164908013CBB
:100E50008A150A128312031964296400831649084B
:100E6000023C8A150A12831203195F286400831654
:100E70004908033C8A110A1283120319C62F640021
:100E800083164908043C8A110A1283120319682F39
:100E9000640083164908053C8A110A12831203195B
:100EA000532F8A01432E8A01E9218A017121831679
:100EB000AA011030AB004C30C50083128A015923BF
:100EC00083164230C40083128A0167218A01432EAF
:100ED0008316F830C700C801B401B501B601B701E7
:100EE00083128A01E9218A0171218316AA01103037
:100EF000AB004C30C50083128A015923831642305F
:100F0000C40083128A01672183165108C200013090
:100F1000B400B5018312831634088312A00083162F
:100F200035088312A100A30120308A01D8208A113C
:100F30000A12031DC42F83160130B600B7018312B5
:100F4000831636088312A000831637088312A10087
:100F5000A30180308A01D8208A110A12031DBB2FF9
:100F60008A015F218316B60A0319B70A8A110A1289
:100F70008312031DA02F8316B40A0319B50A8A1120
:100F80000A128312031D8B2F8A01432E8A01E92145
:100F90008A0171218316AA011030AB004C30C500C4
:100FA00083128A01592383164230C40083128A01B6
:100FB00067218316D90150088312A600A701831662
:100FC0004F088312A200A3018A01ED208316BE0000
:100FD000831225088316BF000130BC00BD018312B7
:100FE00083163C088312A00083163D088312A100DB
:100FF00083163F088312A30083163E0883128A01DA
:10100000D8208A150A12031D5D280730BA00103057
:10101000B8000730BB000830B900A0308A0150206A
:101020007F088A0150207E088A0150208A013520DD
:101030008316C0006400590850028A150A128312F0
:10104000031D412820308316AA070318AB0A463037
:10105000C40083128A01672183162A08C200831202
:101060008A015F2183162B08C20083128A015F2147
:1010700083164C30C40083128A0167218316D9017C
:10108000831283164230C40083128A0167218316BB
:101090004008831288008710000087148316D90A3D
:1010A0008312FE0A0319FF0A8316BC0A0319BD0A3C
:1010B0008A110A128312031DF02F8A01432E831610
:1010C000BE01BF01831211308A012F2011308A0125
:1010D0002F2011308A012F20E830AC000330AD0002
:1010E0008A0105208A110A12031C432E5D3C8A15D1
:1010F0000A12031D7028831641088312A9000530C7
:10110000B000B101A5013C308A0199208A110A1270
:10111000031C432E13308A012F2013308A012F2005
:1011200013308A012F208316C6018312FF308316E5
:1011300041078312B200FF300318013EB30083164B
:1011400046088312A000A1013308A30032088A01D7
:10115000D8208A150A12031DEC28831646083C3E47
:10116000840000088312B200FF30A200A20A220805
:101170000F3C8A150A12031CE0288A150A12CC209B
:1011800032028A150A12031DB62822088316CE00E1
:1011900083128A150A12E02808308A002208820782
:1011A0003034313432343334343435343634373403
:1011B0003834393441344234433444344534463489
:1011C000831646083C3E84004E088000C60A8A15F5
:1011D0000A128312031D96288316C6018312FF305C
:1011E000831641078312B200FF300318013EB3009B
:1011F000831646088312A000A1013308A300320819
:101200008A01D8208A150A12031D6129831646080F
:101210003C3E840000088312B2003208A000A10105
:1012200004308A01D320B2002108B30001308316B4
:1012300046078312B400B501B50D34083C3E840066
:101240000008B400340832048316C2000730831249
:10125000BA001030B8000730BB000830B900A03029
:101260008A0150207F088A0150207E088A01502080
:101270008316420883128A014E2005308A01B3206A
:10128000FE0A0319FF0A8316BE0A0319BF0A3E08A5
:101290008312A00083163F088312A1007D08A300DB
:1012A0007C088A01DB208A150A12031D59298A014C
:1012B000432E02308316C6078A150A128312031CB6
:1012C000EF288A150A1263288A0171218316F830E3
:1012D000C700C801B401B501B601B701D901DA01EF
:1012E000003051078312B20010300318013EB300E2
:1012F000831652088312A600A7012030A200A30182
:101300008A01ED20B4002508B500320834078316A1
:10131000AA00831233080318013E35078316AB0079
:101320004630C40083128A01672183162A08C2004E
:1013300083128A015F2183162B08C20083128A015F
:101340005F2183164C30C40083128A01672111305B
:101350008A012F2011308A012F2011308A012F207D
:10136000B830AC000B30AD008A0105208A110A129A
:10137000031C432E5D3C8A150A12031DB4298316F3
:1013800041088312A9000530B000B101A5013C302D
:101390008A0199208A110A12031C432E13308A01F4
:1013A0002F2013308A012F2013308A012F2083161B
:1013B000C6018312FF30831641078312B200FF304B
:1013C0000318013EB300831646088312A000A10152
:1013D0003308A30032088A01D8208A150A12031D97
:1013E000302A831646083C3E840000088312B2006F
:1013F000FF30A200A20A22080F3C8A150A12031C21
:10140000242A8A150A12102232028A150A12031D92
:10141000FA2922088316CE0083128A150A12242A7A
:101420000A308A00220882073034313432343334AF
:101430003434353436343734383439344134423442
:101440004334443445344634831646083C3E8400D5
:101450004E088000C60A8A150A128312031DDA2973
:101460008316C6018312FF30831641078312B20030
:10147000FF300318013EB300831646088312A00014
:10148000A1013308A30032088A01D8208A150A1264
:10149000031DA72A831646083C3E840000088312D9
:1014A000B2003208A000A10104308A01D320B200AA
:1014B0002108B3000130831646078312B400B5013A
:1014C000B50D34083C3E84000008B40034083204F2
:1014D0008316C0006400590850028A150A1283124C
:1014E000031D912A20308316AA070318AB0A463041
:1014F000C40083128A01672183162A08C20083125E
:101500008A015F2183162B08C20083128A015F21A2
:1015100083164C30C40083128A0167218316D901D7
:10152000831283164230C40083128A016721831616
:101530004008831288008710000087148316D90A98
:101540000230C6078A150A128312031C332A8A1531
:101550000A12A7298A01432E63008A150A12AC2AAF
:02400E00753FFC
:00000001FF
